:1000000000308A009F2E0000FF00030E8301A6002F
:100010007F08A5000A08AD008A01A50E0408A70004
:100020002008A8002108A9002208AA002308AB0084
:100030002408AC00831383128C308400801E222895
:100040008C1A3B288C308400001C28280C183D2872
:10005000270884002808A0002908A1002A08A20077
:100060002B08A3002C08A4002D088A00260E83006C
:10007000FF0E7F0E09008A116B2C8A11B12D0A1018
:100080008A100A118207FF34FF34FF34FF34FF3433
:10009000FF34FF347F34FF34FF34FF343F34FF3408
:1000A000FF34FF341F34FF34FF34FF340F34FF3488
:1000B000FF34FF340734FF34FF34FF340334FF349C
:1000C000FF34FF340134FF34FF34FF340034FF3495
:1000D000FF347F340034FF34FF343F340034FF34C6
:1000E000FF341F340034FF34FF340F340034FF3446
:1000F000FF3407340034FF34FF3403340034FF345A
:10010000FF3401340034FF34FF3400340034FF3452
:100110007F3400340034FF343F3400340034FF3483
:100120001F3400340034FF340F3400340034FF3403
:10013000073400340034FF34033400340034FF3417
:10014000013400340034FF340034003400347F3490
:100150000034003400343F340034003400341F34A1
:100160000034003400340F340034003400340734D9
:1001700000340034003403340034003400340134DB
:100180000034003400340A108A100A11CA3E0318E1
:100190008A0A820000340034003480340034003491
:1001A0000034C034003400340034E034003400340F
:1001B0000034F034003400340034F83400340034B7
:1001C0000034FC34003400340034FE340034003495
:1001D0000034FF34003400348034FF340034003401
:1001E000C034FF3400340034E034FF3400340034D1
:1001F000F034FF3400340034F834FF340034003479
:10020000FC34FF3400340034FE34FF340034003456
:10021000FF34FF3400348034FF34FF340034C03402
:10022000FF34FF340034E034FF34FF340034F03462
:10023000FF34FF340034F834FF34FF340034FC342E
:10024000FF34FF340034FE34FF34FF340034FF3415
:10025000FF34FF348034FF34FF34FF34C034FF34C4
:10026000FF34FF34E034FF34FF34FF34F034FF3424
:10027000FF34FF34F834FF34FF34FF34FC34FF34F0
:10028000FF34FF34FE34FF34FF34FF34FF34FF34D7
:10029000FF34FF340A148A100A1182070034003434
:1002A00000340034003400340034003400340034AE
:1002B00000345F340034003400340034003400343F
:1002C0000234013402340134003400343E34413409
:1002D0004134413422340034003400341034743456
:1002E0001C34173474341C34173404344234253429
:1002F00012340834243452342134003460345634F7
:1003000049344E3430343034403400340034003416
:100310000034043403340134003400340034003435
:100320003E344134003400340034003400340034AE
:10033000003441343E34003400340034003422347C
:1003400014347F3414342234003400340834083434
:1003500008347F340834083408340034003400345E
:1003600080346034203400340034003408340834DD
:1003700008340834083408340834003400340034B5
:1003800000346634663400340034003440342034A1
:100390001034083404340234013400340A148A104E
:1003A0000A11D53E03188A0A82003E346134513462
:1003B0004934453443343E3400340034003440344E
:1003C00042347F3440340034003442346134513498
:1003D00051344934493446340034223441344934A8
:1003E00049344934493436340034303428342434E0
:1003F000223421347F3420340034473445344534AA
:10040000453445344534393400343E344934493474
:10041000493449344934323400340134013401342C
:1004200071340934053403340034363449344934E2
:100430004934493449343634003446344934493433
:100440004934493429341E34003400340034003433
:100450002434243400340034003400340034803434
:100460006434243400340034003400340834143448
:1004700014342234223441340034003424342434FB
:1004800024342434243424340034003441342234D9
:100490002234143414340834003406340134013462
:1004A000593409340934063400340A108A140A1104
:1004B00082073E34413459345534553459342E343E
:1004C000003460341834163411341634183460345F
:1004D00000347F3449344934493449344E3430345B
:1004E00000343E34413441344134413441342234C7
:1004F00000347F34413441344134413441343E345A
:1005000000347F3449344934493449344134403427
:1005100000347F3409340934093409340134013496
:1005200000343E34413441344934493449343A3456
:1005300000347F34083408340834083408347F34F5
:1005400000340034003441347F344134003400340A
:10055000003430344034413441343F3401340034C9
:1005600000347F34083408341434223441340034E5
:1005700000347F344034403440344034403400341C
:1005800000347F34023404340834043402347F34B9
:1005900000347F34023404340834103420347F347F
:1005A00000343E34413441344134413441343E34EA
:1005B00000340A108A140A11E03E03188A0A8200E5
:1005C0007F340934093409340934093406340034D9
:1005D0003E34413441347134493449343E3440343A
:1005E0007F34093409341934293449344634003409
:1005F0002634493449344934493449343234003496
:100600000134013401347F340134013401340034C5
:100610003F34403440344034403440343F3400347C
:1006200003340C343034403430340C34033400346C
:1006300003341C346034183460341C340334003404
:100640004134223414340834143422344134003414
:100650000134023404347834043402340134003474
:1006600041346134553449345534433441340034D1
:10067000003400347F3441344134003400340034D9
:1006800001342A342C3478342C342A3401340034A4
:1006900000340034413441347F34003400340034B9
:1006A000003404340234013402340434003400349D
:1006B000803480348034803480348034803400341A
:1006C0000A148A140A1182070034003401340334F6
:1006D00004340034003400340034383445344534B4
:1006E000453425347E3400347F3444344434443437
:1006F00044343834003400343834443444344434DA
:1007000044344834003400343834443444344434B9
:1007100044347F3440340034383454345434543402
:100720005434583400340034043404347E340534F2
:1007300005340034003400341834A434A434A43410
:10074000A4347834003400347F3408340834083456
:1007500008347034003400340034003400347A3407
:1007600000340034003400340034803480347A346F
:1007700000340034003400347F341034183424340E
:1007800044340034003400340034003400347F3406
:1007900040340034003400347E340434043478347B
:1007A00004340434783400347E340434043404349F
:1007B00004347834403400343834443444344434D9
:1007C00044343834003400340A148A140A11EB3EDD
:1007D00003188A0A8200F83424342434243424345C
:1007E00018340034003418342434243424342434A9
:1007F000F834003400347C340834043404340434D1
:1008000000340034003448345434543454345434B0
:10081000203400340034043404343F344434443449
:100820000034003400343C3440344034403420340C
:100830007C344034003404341834603430340C34A4
:100840000434003400341C346034183460341834F8
:10085000043400340034443428341034283444340C
:100860004034003400340434883490346034183414
:1008700004340034003444346434543454344C3438
:100880004434003400340034003408343634413405
:100890000034003400340034003400347F34003439
:1008A0000034003400340034003441343634083429
:1008B0000034003400340034003401340234013494
:1008C0000234003400342A3455342A3455342A345E
:1008D00055342A3400348C128A11282887100714C2
:1008E000003487140710003400308316860083120A
:1008F0003208860085100330A000A00B7D2C8511E6
:100900000330A000A00B822C851500000000000021
:100910000000000000340030831686008312300887
:10092000860085140330A000A00B942C85110330A1
:10093000A000A00B992C851500000000000000000D
:1009400000000034871007100034A224C5014508B8
:10095000023C031CBD2C4508B838B2007424C40105
:1009600044083C3C031CBB2C4408B2007424B00176
:100970008B24C40AB02CC50AA72C003449081F3C9C
:100980000318C62C4908803C031CC62C49080F39A3
:10099000A000200DC400C40DC40DF830C4054908E2
:1009A0002F3C031CE42CC5014508073C031CE32C29
:1009B000333045078400831344084A21A100800096
:1009C000C40AC50AD42C4C2D49083F3C031CF92C01
:1009D000C5014508073C031CF82C3330450784004B
:1009E00083134408CE21A1008000C40AC50AE92C63
:1009F0004C2D49084F3C031C0E2DC5014508073CF2
:100A0000031C0D2D33304507840083134408552201
:100A1000A1008000C40AC50AFE2C4C2D49085F3C89
:100A2000031C232DC5014508073C031C222D333030
:100A30004507840083134408D922A1008000C40A1A
:100A4000C50A132D4C2D49086F3C031C382DC501D8
:100A50004508073C031C372D3330450784008313BA
:100A600044086023A1008000C40AC50A282D4C2D2B
:100A700049087F3C031C4C2DC5014508073C031C5D
:100A80004C2D33304507840083134408E423A10030
:100A90008000C40AC50A3D2D3B083C3C031C542D74
:100AA0003B08C4006E24582D3D303B02C400712425
:100AB0003B08783C03185E2DBB01BC0A3C08033C94
:100AC000031CBC01C5014508073C031C7F2D3C08E5
:100AD000B838B20074244408B20074243330450797
:100AE000840083130008B0008B24BB0AC40A3B08AF
:100AF0003D3C031D7D2DC4017124C50A632D0034C6
:100B0000BB013B08BC006E24B830B2007424B201B3
:100B100074241830BB004E30C900BE246530C900B3
:100B2000BE246F30C900BE242D30C900BE2454300D
:100B3000C900BE246530C900BE246330C900BE248C
:100B40006830C900BE242D30C900BE244C30C90015
:100B5000BE246130C900BE246230C900BE24BB017E
:100B600000343C308F00AF308E00C30A4308023C93
:100B70000318902EC3011F151F19BC2D83161E08C4
:100B80008312C9001E0CA300490CA200A30CA20CE6
:100B9000A30CA20CA30CA20CA30CA20C2208BD0057
:100BA0003D083E020318162E3E0DA000A00DFC309D
:100BB000A0052008C9000330C90749083F20A30049
:100BC000C90349083F20A200C90349083F20A100EA
:100BD00049033F20A0002308CD002208CC002108B3
:100BE000CB002008CA003D0DA000A00DFC30A005E0
:100BF0002008CE000330CE074E08C320A300CE034A
:100C00004E08C320A200CE034E08C320A1004E030D
:100C1000C320A0004A05BF0021084B05C0002208E0
:100C20004C05C10023084D05C200572E3D0DA00004
:100C3000A00DFC30A0052008C9000330C9074908F1
:100C40003F20A300C90349083F20A200C903490867
:100C50003F20A10049033F20A0002308CD00220827
:100C6000CC002108CB002008CA003E0DA000A00D3A
:100C7000FC30A0052008CE000330CE074E08C3206C
:100C8000A300CE034E08C320A200CE034E08C3200B
:100C9000A1004E03C320A0004A05BF0021084B0558
:100CA000C00022084C05C10023084D05C2003B08C6
:100CB0003C3C031C5F2E3B08C4006E24632E3D3079
:100CC0003B02C4007124B830B20074244408B2005E
:100CD00074243F08B0008B24B930B2007424440857
:100CE000B20074244008B0008B24BA30B2007424DF
:100CF0004408B20074244108B0008B24BB30B20019
:100D000074244408B20074244208B0008B24BB0A47
:100D10003B087A3C031D8E2EA52480253D08BE008D
:100D20000C108A112828A224AF30B20074248A1132
:100D3000E72EA224C030B20074248A11E82E840168
:100D400083131F30830583161F149F141F159F11D3
:100D50004030990026309800903083129800831616
:100D600081170030860038308312850001308316E9
:100D700085004330831287009030831687008312EA
:100D800007110C3097000030A10006389200FF30A8
:100D9000831692007F30831295001708CF393038C0
:100DA00097001F139F1783169F1783121F14831614
:100DB0001F109F141F159F1500308312A1001F08DC
:100DC000C73921049F00EE30B2007424932E992E6F
:100DD000AE018B1BAE178B13A524AE1B8B17AE0178
:100DE0008B1BAE178B138025AE1B8B17BE013E08E5
:100DF000BD00853090003C308F00AF308E00C301C5
:0E0E000083160C14C03083128B04052F630080
:02400E003A3F37
:00000001FF
